:020000040800F2
:10000000000200207904000809220008AD21000840
:10001000ED210008AD210008CD2100087B04000877
:100020007B0400087B0400087B040008BD30000846
:100030007B0400087B0400087B040008B13C000836
:100040007B0400087B0400087B0400087B04000894
:100050007B0400087B040008E5390008113A000819
:100060003D3A0008693A0008953A00087B04000808
:100070007B0400087B0400087B0400087B04000864
:100080007B0400087B0400087B040008F51D0008C1
:10009000211E0008311E00087B040008C13A000838
:1000A0007B0400087B0400087B0400087B04000834
:1000B0007B0400087B0400087B0400087B04000824
:1000C0007B0400087B0400087B0400087B04000814
:1000D0007B0400087B0400087B0400087B04000804
:1000E000293B00087B0400087B0400087B0400080F
:1000F0007B0400087B0400087B0400087B040008E4
:100100007B0400087B0400087B0400087B040008D3
:100110007B0400087B0400087B0400087B040008C3
:100120007B0400087B0400087B0400087B040008B3
:100130007B0400087B0400087B0400087B040008A3
:100140007B0400087B0400087B0400087B04000893
:100150007B0400087B0400087B0400087B04000883
:100160006112000800000000000000000000000014
:1001700053B94AB9002908BF00281CBF4FF0FF310E
:100180004FF0FF3000F076B9ADF1080C6DE904CE08
:1001900000F006F8DDF804E0DDE9022304B0704762
:1001A0002DE9F047089E0D4604468846002B4DD1A8
:1001B0008A42944668D9B2FA82F252B101FA02F345
:1001C000C2F1200120FA01F10CFA02FC41EA030815
:1001D00094404FEA1C41B8FBF1F71FFA8CFE01FB7B
:1001E000178807FB0EF0230C43EA084398420AD90C
:1001F0001CEB030307F1FF3580F01E81984240F2AB
:100200001B81023F63441B1AB3FBF1F001FB103367
:1002100000FB0EFEA4B244EA0344A6450AD91CEB37
:10022000040400F1FF3380F00981A64540F2068105
:10023000644402380021A4EB0E0440EA07401EB1DA
:100240000023D440C6E90043BDE8F0878B4208D9BB
:10025000002E00F0EE800021C6E900050846BDE84A
:10026000F087B3FA83F100294AD1AB4202D382422C
:1002700000F2FC80841A65EB030301209846002EEF
:10028000E2D0C6E90048DFE702B9FFDEB2FA82F247
:10029000002A40F09180A1EB0C0001214FEA1C479D
:1002A0001FFA8CFEB0FBF7F307FB1300250C45EAA1
:1002B00000450EFB03F0A84208D91CEB050503F12D
:1002C000FF3802D2A84200F2CE8043462D1AB5FB79
:1002D000F7F007FB10550EFB00FEA4B244EA0544FC
:1002E000A64508D91CEB040400F1FF3502D2A6454F
:1002F00000F2B6802846A4EB0E0440EA03409EE7D5
:10030000C1F120078B4022FA07FC4CEA030C25FAC6
:1003100007FA4FEA1C49BAFBF9F820FA07F309FB80
:1003200018AA8D401FFA8CFE1D4300FA01F308FB4A
:100330000EF02C0C44EA0A44A04202FA01F20BD956
:100340001CEB040408F1FF3A80F08880A04240F2E0
:100350008580A8F102086444241AB4FBF9F009FB73
:10036000104400FB0EFEADB245EA0444A64508D990
:100370001CEB040400F1FF356CD2A6456AD90238A3
:10038000644440EA0840A0FB0295A4EB0E04AC4292
:10039000C846AE4656D353D0002E69D0B3EB080200
:1003A00064EB0E0422FA01F304FA07F71F43CC4072
:1003B000C6E90074002147E70CFA02FCC2F12001F3
:1003C00025FA01F34FEA1C4720FA01F195400D434D
:1003D000B3FBF7F107FB11331FFA8CFE280C40EA40
:1003E000034001FB0EF3834204FA02F408D91CEB2C
:1003F000000001F1FF382FD283422DD90239604429
:10040000C01AB0FBF7F307FB1300ADB245EA004595
:1004100003FB0EF0A84208D91CEB050503F1FF38D9
:1004200016D2A84214D9023B6544281A43EA014176
:1004300038E73146304607E72F46E4E61846F9E646
:100440004B45A9D2B9EB020865EB0C0E0138A3E7C6
:100450004346EAE7284694E74146D1E7D0467BE7A2
:100460006444023847E7023B65442FE7084606E745
:100470003146E9E6704700BF02E000F000F8FEE711
:1004800072B6284880F30888274880F309882748EF
:100490004EF60851CEF200010860022080F3148865
:1004A000BFF36F8F03F026FA03F002FA03F024FA89
:1004B0004FF055301E491B4A91423CBF41F8040B96
:1004C000FAE71C49184A91423CBF41F8040BFAE78D
:1004D00019491A4A1A4B9A423EBF51F8040B42F886
:1004E000040BF8E700201749174A91423CBF41F836
:1004F000040BFAE703F0E0F903F000FA134C144D93
:10050000AC4203DA54F8041B8847F9E700F03CF8E2
:10051000104C114DAC4203DA54F8041B8847F9E73C
:1005200003F0C8B900020020000800200000000805
:10053000000100200002002068410008000800209F
:1005400080080020800800206C2000206001000846
:100550006401000864010008640100082DE9F04FFF
:10056000C1F80CD0C3689D46BDE8F08F002383F32B
:1005700011882846A047002002F048FFFEE702F05D
:10058000C1FE00DFFEE700002DE9F0412F4A53686D
:1005900023F0E06343F0905343F48043536003F04F
:1005A00021F9074603F070F90546B8BB284B9F4276
:1005B00034D001339F4234D0264B27F0FF029A42B9
:1005C00033D1F8B200F066FAA84642F2107400F097
:1005D0006BFC08B10024A04600F062FA064640B366
:1005E0004CBB464635B11C4B9F4203D0002403F060
:1005F00043F92646002003F0FFF80EB100F02EF874
:1006000000F0B0FC00F03EFE01F006FE0546ACB97D
:1006100000F0EEFC012002F0FFFEF8E7A8460024FF
:10062000D5E704464FF00108D1E7804641F288340F
:10063000CDE70446D6E74FF47A74D3E701F0ECFD3A
:10064000431BA342E4D900F009F8DDE700000140B4
:10065000010007B0000008B0263A09B038B51D4ABD
:100660001D4B1968013134D004339342F9D11B4C2E
:10067000194DD4F80428AA422BD3194B9B6803F1D7
:10068000006303F508439A4223D203F0C9F803F04C
:10069000DBF8002000F01CFE0220124B187000F066
:1006A00053FE114BDA690022DA61D96999699A61BE
:1006B0009B6972B64FF0E023C3F8085DD4F80038A8
:1006C000D4F80428202181F311889D4683F30888FB
:1006D000104738BD20880008008800080080000806
:1006E00000080020800800200010024049F2690044
:1006F000084A136899B21B0C00FB013344F25061A5
:100700001360054B186882B2000C01FB02001860F0
:1007100080B27047180800201408002010B5044665
:100720000021102200F02CFE034B03CB20606160FF
:100730001868A06010BD00BFE8F7FF1F2DE9F04367
:10074000BBB001F069FD40F2ED22204DAB68C31A49
:10075000934232D906AF2B4628220021A8603846A2
:1007600002F066FA05F10E0000F002FE00260446D3
:100770005FFA80F905F10E08F3B2F100994501F135
:10078000280107D908EB06030822384602F050FA80
:100790000136F1E708230122CDE902320C4B053482
:1007A00001933023A4B20093CDE9047405A3D3E9E7
:1007B0000023297B074802F051F83BB0BDE8F083E5
:1007C000AFF3008078F6339F93CACD8D981D00203B
:1007D000A51D00209C18002070B50D4614461E462D
:1007E00001F0D2FF50B9022E10D1012C0ED112A36C
:1007F000D3E900230120C5E9002307E0282C10D00D
:1008000005D8012C09D0052C0FD0002070BD302C4C
:10081000FBD10BA3D3E90023ECE70BA3D3E900231F
:10082000E8E70BA3D3E90023E4E70BA3D3E9002314
:10083000E0E700BFAFF30080401DA12026812A0B16
:1008400078F6339F93CACD8D9E6AC421818A46EE85
:1008500026417272DF25D7B7F017304A39059E5608
:1008600038B50D460446034620222846002102F0F2
:10087000DFF922792346032A28BF0322284603F8FA
:10088000042F2021022202F0D3F962792346072A9D
:1008900028BF0722284603F8052F2221032202F051
:1008A000C7F9A2792346072A28BF0722284603F85A
:1008B000062F2521032202F0BBF928461022282109
:1008C00004F1080302F0B4F9382038BD2DE9F04FE7
:1008D0000024ADF5037D10AE40F2751280460F4640
:1008E00024A82146239400F04BFD2146482230469F
:1008F00000F046FD01F090FC4FF47A72B0FBF2F08C
:10090000544B23AD186093E80700012386E80700E5
:100910000DF162003382FFF701FF4EF6035333847B
:1009200007AB18464C4903F039FB212229463064B5
:10093000304686F83C20FFF793FF08220446014624
:1009400014AB284602F074F908222846A1180DF1CC
:10095000510302F06DF9082228460DF1520304F10B
:10096000100102F065F92022284615AB04F11801A8
:1009700002F05EF94022284616AB04F1380102F07D
:1009800057F90822284618AB04F1780102F050F913
:10099000082228460DF1610304F1800102F048F9B4
:1009A00004F1880A0DF1620904F5847B4B46514637
:1009B000082228460AF1080A02F03AF9D34509F15B
:1009C0000109F3D10822594628461DAB02F030F93F
:1009D0004FF0000904F5887496F834304B450AD975
:1009E000B36B21464B440822284602F021F9083413
:1009F00009F10109F0E74FF0000996F83C3004EBEB
:100A0000C9014B4508D9336C08224B44284602F0F3
:100A10000FF909F10109F0E700230393BB7E0731C9
:100A2000029307F1190301930123C1F3CF01CDE92B
:100A300004510093404605A3D3E90023F97E01F059
:100A40000DFF0DF5037DBDE8F08F00BF9E6AC42148
:100A5000818A46EE84080020CC3F000810B50A4B7E
:100A60000A4A1A6093F8602442B9D3F85C442CB166
:100A7000204601F067FA204603F028F9BDE810404F
:100A8000034801F05FBA00BFC8180020B440000856
:100A9000101D0020014B1870704700BF9008002007
:100AA000F0B5334B85B01C7B34B10E22314B1A812B
:100AB0000024204605B0F0BD2F4A02AB10685168F3
:100AC00003C308232D492E480DEB030203F050F910
:100AD000054630B90A22274B2A481A8101F0B0F99D
:100AE000E6E70169B1F55E3F06D90B22214B2648A6
:100AF0001A8101F0A5F9DCE740F2ED32438B934215
:100B000007D00C201B4908811946204801F098F9AC
:100B1000CFE71F4A024402F11003994204D2102287
:100B2000144B1C481A81E4E710398E1A20461449E8
:100B300001F078FB07463246204605F1180101F026
:100B400071FBAB689F4202D1EB6898420AD00D223C
:100B5000084B1A8100903B46D5E902120E4801F07D
:100B60006FF9A5E70D4801F06BF90124A1E700BF7B
:100B7000981D00208408002081400008DC770300D5
:100B800000880008F03F0008FC3F00080E40000805
:100B90000878FFF72C400008494000087240000820
:100BA0002DE9F04FADB006AF80460C4601F0ECFDEC
:100BB0000546002859D1237E022B1AD1E38A012B46
:100BC00017D101F029FB0646FFF790FD4FF4C873DB
:100BD000B0FBF3F202FB1300DFF8B49206F51676D1
:100BE00080B2E37E0644C9F8006033B90022A94B05
:100BF0001A709C37BD46BDE8F08FA38AEEB2013B68
:100C0000B34205F101050BD93B1D1E44E900002349
:100C100008222046009601F0F80101F0CBFEECE737
:100C200007F11400FFF77AFD324607F11401381D71
:100C300003F08EF803460028D8D10F2E08D8954B24
:100C40001E70D9F80030A3F51673C9F80030D0E74C
:100C5000FA1CF870014600922046072201F0AAFE15
:100C60004046F97801F088FDC3E7E38A282B26D0B7
:100C700010D8012B1ED0052BBBD1BFF34F8F864957
:100C8000864BCA6802F4E0621343CB60BFF34F8F18
:100C900000BFFDE7302BACD1637E814D01336A7B11
:100CA000DBB29342E94603D1E27E2B7B9A4265D0C8
:100CB000CD469EE721464046FFF708FE99E7A38A06
:100CC000013B9BB2C92B94D8754D2E7B26BB05F1F9
:100CD0000C030093082233463146204601F06AFE99
:100CE000731CF2B2D9001E46A38A013B9A4205DA70
:100CF0000E322A44009200230822EEE7002300224D
:100D0000C5E900230023AB6085F8D730C5F8D8309B
:100D10002B7B0BB9E37E2B73002507F11406082209
:100D2000294630463B1DC7E90155FD6001F080FFB3
:100D30003B7A05F10109AB424FEAC90107D9FB68CB
:100D400008222B44304601F073FF4D46F0E70023A4
:100D5000C1F3CF01E07ECDE904610393A37E193492
:100D60000293282301460093404647A3D3E900237A
:100D7000019401F073FDFFF7E1FC3AE74FF0000842
:100D800007F11403A7F814801022009341460123B1
:100D9000204601F00FFEA68A023EB6B2F31C9B105D
:100DA0009B000733DB08A9EBC3039D460DF1180A2E
:100DB0001FFA88F34FEAC801B34201F110010AD2C9
:100DC0000AEB0803009308220023204601F0F2FDFD
:100DD00008F10108ECE795F8D70000F083FAD5F8A0
:100DE000D83004461BB995F8D70000F08BFAD5F837
:100DF000D83033449C4204D295F8D700013000F03B
:100E000081FA4FF000084FEA960B1FFA88F18B45E4
:100E1000D5E9003209D90AEB880103EB88000122E9
:100E200000F0B6FA08F10108EFE7F31842F100020A
:100E3000C5E90032D5F8D83095F8D70006EB03089D
:100E4000C5F8D88000F04EFA804509D395F8D73020
:100E5000D5F8D8000133001B85F8D730C5F8D80085
:100E6000FF2E08D800232B7300F05EFAFFF718FE60
:100E700008B1FFF7F3FB2B680A4A9B0A0133138181
:100E80000023AB6014E700BF26417272DF25D7B79D
:100E9000981800209518002000ED00E00400FA05E5
:100EA000981D00208408002030B54FF00054244BDA
:100EB000226885B09A4207D002F0F0FC0446A8B937
:100EC0000024204605B030BD627D1E4B1E481A70BE
:100ED000237DC92203731D490E3000F03FFA2046DE
:100EE000E022002100F04CFA0124EAE7184A194DEB
:100EF000D36943F00073D361AA6D174B9A42DFD1D7
:100F00002B6E013B7E2BDBD8144A01AB07CA83E86A
:100F100007001846032101F09BF96B6D83424FF0E7
:100F20000003CDD12A6D8A4203BFAB652A6E054B03
:100F30001C4601BF1A70EA6D094B1A60C1E700BF79
:100F40009AAD44C590080020981D0020160000208E
:100F500000100240006600405041A0B058660040BA
:100F600010080020022337B5184D01226B71184B71
:100F70001848196800F036FE00230193164B1749F4
:100F800000934FF48052164B164801F0CDFB164BE0
:100F9000197811B1134801F0EFFB01F03DF9044657
:100FA000FFF7A4FB4FF4C873B0FBF3F202FB13038B
:100FB00004F516709BB218440C4B186002F064FCE8
:100FC00008B10F232B8103B030BD00BF840800207F
:100FD00010080020C8180020D90700089408002035
:100FE000A10B00089C1800209008002098180020F1
:100FF0002DE9F04F0FF26029D9E900898A4C93B0AE
:101000008A4E8B4F204601F08DFC034660B30025CD
:10101000CDE90F550E95ADF84450027BDFF814A2D0
:101020008DF84420996840680FAA03C21B6843F0FA
:1010300000430E9301F0F2F8821941F100033846A3
:1010400000950EA900F014FAA84205DD204601F033
:101050006DFC8AF80050D5E79AF80030072B00F2B3
:10106000B78001338AF8003000230BAE704FDFF8F1
:10107000C8A10A93ADF834300B9373604FF0000BA6
:10108000002200230125CDE9002338465B460DF1FF
:101090001D0207A98DF81C508DF81DB000F054FDFD
:1010A0009DF81C30002B40F09780204601F06CFB2F
:1010B0000646002848D101F0AFF8DFF880A1DAF841
:1010C0000030984240D301F0A7F80746FFF70EFB27
:1010D0004FF4C873B0FBF3F202FB130007F5167769
:1010E00080B20744CAF80070554F0EA897F800B0B8
:1010F000BBF1000F14BF33462B46CBF1100A5FFA49
:101100008AFA8DF82830FFF709FBBAF1060F28BFDD
:101110004FF0060A0EAB03EB0B0152460DF129000E
:1011200000F01CF90AAB039318230AF101020293A1
:10113000444BD2B2CDE900530492204638A3D3E900
:10114000002301F023FB3E7001F066F83E4A3F4D5C
:101150001368C31AB3F57A7F2FD3106001F05EF8DD
:1011600002460B46204601F0EBFB204601F00CFB4B
:1011700018B32B7B364E002B14BF0323022373714D
:1011800001F04AF84FF47A73B0FBF3F00EAF306021
:1011900039463046FFF764FB182302932D4B073086
:1011A000019340F25513C0F3CF00CDE903700093D3
:1011B00042464B46204601F0E9FA2B7B2BB1FFF764
:1011C000BDFA2B7B002B7FF41BAF13B0BDE8F08F73
:1011D000204601F0ABFB47E7DAF80C30594683F0C4
:1011E0000803CAF80C3010220EA800F0C9F80DF15F
:1011F0001E0308AA0AA9384600F032FA96E803004E
:101200000FAB83E803009DF8343020468DF844305E
:101210000A9B0EA90E93DDE9082301F051FD2DE78D
:10122000401DA12026812A0B9C18002040420F005F
:10123000C81800207D1E0020000C014098180020D6
:101240009518002094180020781E0020981D00207A
:10125000840800207C1E0020F1C6A7C1D068080FBA
:1012600008B5054800F092FABDE808400020034A9E
:10127000034902F025BD00BFC8180020B81E002099
:101280005D0A000870B502F07DF900250E4C0F4E86
:1012900020803068238883420CD8002520880138BC
:1012A00002F06CF923880544013BB5F5805F23808B
:1012B000F4D370BD02F062F9336805440133B5F52B
:1012C000084F3360E5D3E8E7AC1E0020801E002005
:1012D00002F0F6B900F10060920000F5084002F05B
:1012E00091B90000054B1A68054B1B889B1A834275
:1012F00002D9104402F042B900207047801E00203D
:10130000AC1E002038B50446064D2868204402F083
:101310003BF928B928682044BDE8384002F046B9B6
:1013200038BD00BF801E0020064991F8243033B13B
:1013300000230822086A81F82430FFF7CBBF012080
:10134000704700BF841E0020022802BF4FF4002215
:10135000014B1A61704700BF000C0140002310B51B
:10136000934203D0CC5CC4540133F9E710BD0000B4
:1013700003460246D01A12F9011B0029FAD1704720
:1013800003460244934202D003F8011BFAE7704778
:101390002DE9F8431F4D144695F82420074688464A
:1013A00052BBDFF870909CB395F824302BB9202203
:1013B000FF2148462F62FFF7E3FF95F824004146DE
:1013C000C0F10802A24228BF224605EB8000D6B237
:1013D0009200FFF7C3FF95F82430A41B1E44F6B219
:1013E000082E17449044E4B285F82460DBD1FFF75F
:1013F0009BFF0028D7D108E02B6A03EB82038342CE
:10140000CFD0FFF791FF0028CBD10020BDE8F883B3
:101410000120FBE7841E0020202383F3118862B69D
:1014200070470000002383F3118862B67047000004
:1014300010B4026854681A46234610BC18470000CE
:10144000012070470020704700207047704700005F
:1014500070470000002070470E20704790F8C804C5
:10146000C0F340007047000090F9C90470470000C5
:101470002DE9F0410C681E4614F00054BDF81870B8
:101480006AD10B7B082B67D8FFF7C6FF4569AB68AD
:101490005B010CD4AB681B0108D4AC6814F0805419
:1014A00058D1FFF7BFFF2046BDE8F08101240B684B
:1014B00004F1180C002BBABFDB0043F004035B05FA
:1014C0004FEA0C1C45F80C300B684FEA041C13F073
:1014D000804F1CBF05EB0C0EDEF88031AC441CBF06
:1014E00043F00203CEF880310B7B05EB0415CCF8FA
:1014F00084318B68C5F88C314B68C5F888310D464E
:10150000DCF8803143F00103CCF8803100EB441368
:10151000C3F86824C3F86C6401F10C0C03F58E6306
:1015200055F804EB654543F804EBF9D12D882434D4
:101530001D8000EB4414257907F0030325F00B050B
:101540002B432371FFF76EFF33460697BDE8F0414A
:1015500000F098BC0224AAE74FF0FF30A4E7000097
:1015600038B50446D0F85C040D4600F01FFD1F2876
:101570000AD920222946D4F85C0400F08DFDA0F1A0
:1015800020035842584138BD0020FCE708B5FFF75A
:1015900043FFD0F85C0400F0DFFCBDE80840FFF733
:1015A00041BF000000220260828142608260704779
:1015B0000022002310B5C0E9002300230446038164
:1015C0000C30FFF7EFFF204610BD0000F0B590F89B
:1015D000C8340D4613F0040FC3F3800108BF114651
:1015E00005F1240661F3820380F8C83400EB46134A
:1015F0001B790446D80789B02DD572B319072CD4AE
:1016000004EB45156846FFF7D3FF05F58E6303AA83
:1016100005F58F65174618685968083303C7AB424C
:101620003A46F7D11868694638609B882046BB80E7
:10163000DDE90E23CDE900230123ADF8083023684E
:101640001B6C984704EB461423791A075CBF43F0E0
:101650000803237101E0002AF4D109B0F0BD0000B5
:101660002DE9F047054688B068469A468846914677
:10167000FFF7D2FEFFF79CFFD5F85C0400F07EFC7C
:101680001F282AD920226946D5F85C0400F082FD83
:10169000202822D1444603AE05AB374603CF9F42F4
:1016A000206061603E4604F10804F6D13868414686
:1016B0002060BB882846A380DDE90023C9E9002318
:1016C000BDF808304A46AAF80030FFF7ABFE534693
:1016D00008B0BDE8F04700F0C3BB0020FFF7A2FE52
:1016E00008B0BDE8F087000000232DE9F04704466C
:1016F000C0E90133224B0E4640F8183BFFF752FF7A
:1017000004F1480704F12800FFF752FF3D4604F5B5
:10171000896828462035FFF74BFF4545F9D14FF43E
:101720008063C4F84874C4F84C34002701234FF098
:1017300000084FF00009C4F85C54C4F85074C4F8B1
:10174000547484F8583484F8603404F5916504F5D1
:101750009D6A45E90889A5F11800FFF723FF2035A8
:1017600045F8287C5545F4D184F8C96416B105487C
:1017700000F04CFD044B20466361BDE8F08700BFDC
:10178000B44000088C4000080064004010B50446D6
:10179000034B19784A1C1A70FFF7A6FF204610BDAC
:1017A000B41E00202DE9F04300294FD0284F294BCB
:1017B000B7FBF1F499428CBF0A231123B4FBF3FC6D
:1017C000581E03FB1C43C5B22BB102280346F5D8B3
:1017D0000020BDE8F0830CF1FF36B6F5806FF7D23C
:1017E0004FF47A74C5EBC50E0EF103034FEAE3091B
:1017F00009FB0444C3F3C703E81AC0B209F10108A6
:101800008044B4FBF8F4B4F5617FC2BF0EF1FF333E
:10181000C3F3C703E81A03F10104C8BFC0B2E4B2BE
:1018200004440CFB04F4B7FBF4F4A142D0D1013B17
:10183000DBB20F2BCCD80138C0B20728C8D80021A2
:101840001071168001209170D370C2E70846C0E77E
:10185000005125023F420F0070B505460E464FF479
:101860007A746B6901205B6803F00103B34204D012
:1018700001F0D2FD013CF4D1204670BD30B5426983
:10188000936913F0700F16D000230B4C936103F192
:10189000240200EB421211794D0709D5890707D5BB
:1018A000416954F823508D60117941F004011171A0
:1018B0000133032BEBD130BDA040000873B51D46AA
:1018C000436916469A680446D20709D501219A68E9
:1018D0009960C2F340020021CDE90065FFF776FE72
:1018E00063699A68D1050BD54FF480719A682046D8
:1018F0009960C2F340220121CDE90065FFF766FE41
:1019000063699A68D2030BD54FF480319A682046F8
:101910009960C2F340420221CDE90065FFF756FE0F
:10192000204602B0BDE87040FFF7A8BFF8B50446F6
:10193000466900296AD106F10C073868800768D02B
:10194000386806EB01104FEA011CD0F8B011D0F84E
:10195000B051490746BFED0845F000456D0DA56142
:10196000D0F8B011890744BF45F08045A561D0F893
:10197000B40106EB0C0100F00F0084F82400D1F84C
:10198000B80104F124052077D1F8B801000A607786
:10199000D1F8B801000CA077D1F8B801000EE077BB
:1019A000D1F8BC0184F82000D1F8BC01000A84F809
:1019B0002100D1F8BC01000C84F82200D1F8BC1140
:1019C00004F13400090E84F823103821396004F141
:1019D000180151F8046BA94240F8046BF9D1098849
:1019E0000180C4E90A2300232146238651F8283BBD
:1019F00020461B6C984794F8C834204643F00403F3
:101A000084F8C834BDE8F840FFF738BF06F1100786
:101A100093E7F8BD10B5044600F000FC02460B4603
:101A200052EA030102D0013A63F100030449086855
:101A300020B12146BDE81040FFF778BF10BD00BFC0
:101A4000B01E0020F8B500211E46FFF7E5FC124F3E
:101A500000F58D6501F1240400EB4414237913F0A3
:101A6000040F0FD1DB060DD5D5E900C39445B34172
:101A700008D2436957F821C0C3F808C0237943F05E
:101A8000040323710131032905F12005E2D1BDE8EA
:101A9000F840FFF7C7BC00BFA040000808B5FFF73B
:101AA000BBFCFFF7EBFEBDE80840FFF7BBBC000046
:101AB000F8B54369044698680E4600F0E050B0F16E
:101AC000E05F1DD0D8B1FFF7A7FC002504F58E67B5
:101AD00004EB451393F884341A0706D50135032D1A
:101AE00007F12007F4D1012007E05B07F6D439465F
:101AF000304600F001FA0028F0D1FFF793FCF8BD62
:101B00000120FCE708B5FFF787FCD0F85C0400F083
:101B100035FAFFF787FC43090CBF0120002008BD00
:101B2000F8B51D46002313700F4606461446FFF70E
:101B3000E9FF80F00100387025B129463046FFF7F3
:101B4000B7FF2070F8BD0000F8B50C4615461E46DC
:101B5000074600F063FB0B462178024609B9287856
:101B600050B13846FFF76EFFFFF798FF33462A461D
:101B70002146FFF7D5FF0120F8BD000010B5FFF7A3
:101B80004BFC174B0446DA6942F00072DA611A69BD
:101B900042F000721A611A6922F000721A61FFF7AE
:101BA00041FC90F8C834DB0718D4B9B102211320E6
:101BB000FFF732FC01F0D2FA0221142001F0CEFA34
:101BC0000221152001F0CAFA94F8C83443F0010349
:101BD00084F8C834BDE81040FFF724BC10BD00BF36
:101BE000001002402DE9F04790F8C9340446012B5B
:101BF0000F46154688B000F2F9807D4E56F8232036
:101C00000AB946F82300D6F80090E7602574B9F1C8
:101C1000000F09D14FF49A6002F05AF88046494605
:101C2000FFF762FDC6F8008094F8C934012B5CD040
:101C30004FF0000801212046FFF7A0FFFFF7ECFB63
:101C4000626901211368204623F002031360626970
:101C5000136843F0010313606369C3F81480FFF74E
:101C6000E1FBFFF7F9FD002800F08180D4F85C0467
:101C700000F072F9A14604F1600A202200216846B2
:101C8000FFF77EFB02A8FFF78DFC6A46CDF81880AF
:101C900009F58D630DF1180C164603CE66451860E4
:101CA0005960324603F10803F6D1306809F1200982
:101CB00018603279CA451A71DFD1002694F8C83409
:101CC0006A466FF3820384F8C83439462046ADF87B
:101CD0000060ADF802608DF80460FFF763FD636992
:101CE000C0B94FF400421A6011E0306803685B6BC2
:101CF0009847014600289BD13068FFF73FFF3068C6
:101D00002A46036839465B689847002890D108B096
:101D1000BDE8F0876122022D0CBF4FF00041002189
:101D20001A609DF802309DF803201B06120402F48D
:101D3000702203F040731343BDF800202046C2F325
:101D4000090213439DF80420120502F4E002134334
:101D500062690B43D3611322636931465A61626938
:101D6000136823F001031360FFF776FD08B9636978
:101D7000B7E794F8C93493BB6169D1F8002242F007
:101D80000102C1F800226169D1F8002222F47C52DC
:101D900022F00E02C1F800226169D1F8002242F45B
:101DA0006062C1F8002241F6FF716269C2F8143224
:101DB0006269C2F804326269C2F80C126269C2F840
:101DC00040326269C2F8443201226369C3F81C22BE
:101DD0006269D2F8003223F00103C2F8003294F8AD
:101DE000C83443F0020384F8C83490E700208EE73B
:101DF000B01E002008B500F011FA02460B4652EA68
:101E0000030102D0013A63F100030449086808B1F4
:101E1000FFF754FDBDE8084001F07EB9B01E002078
:101E200008B50020FFF7F6FDBDE8084001F074B9E1
:101E300008B50120FFF7EEFDBDE8084001F06CB9E0
:101E40000FB4002004B0704713B56C4684E8060058
:101E5000031D94E8030083E80500012002B010BDD3
:101E6000F8B586680D4656B11B885B0707D4D0E9E4
:101E70000037DB6B98472A46C1B23846B04701208D
:101E8000F8BD0000F0B5866805460C4689B05EB125
:101E9000BDF838305B070AD4D0E90037DB6B9847D0
:101EA0002246C1B23846B047012009B0F0BD002239
:101EB0000023CDE9002300230A46ADF8083001F1E4
:101EC000080603AB1C4610685168083203C4B242CE
:101ED0002346F7D1106820609288A28000F0A0F914
:101EE0000423ADF808302B68CDE900011B6C69466E
:101EF00028469847D8E7000030B503680968DD0F29
:101F0000B5EBD17F23F0604421F060424FEAD170FD
:101F10000BD0002BB8BFA40C0029B8BF920C944280
:101F200002D034BF0120002030BD944205D1C1F35E
:101F30008070C3F380738342F6D194422CBF00209B
:101F40000120F1E710B5037C044613B9006801F0E5
:101F5000F7FE204610BD00000023BFF35B8FC36077
:101F6000BFF35B8FBFF35B8F8360BFF35B8F704703
:101F7000BFF35B8F0068BFF35B8F704770B505469A
:101F80000C30FFF7F5FF05F1080604463046FFF771
:101F9000EFFFA04206D930466D68FFF7E9FF2C44F9
:101FA000201A70BD3046FFF7E3FFF9E770B505462C
:101FB0004068A0B105F10800FFF7DAFF05F10C0653
:101FC00004463046FFF7D4FF844288BF00253046E0
:101FD00098BF6D68FFF7CCFF013C2C44201A70BD00
:101FE00038B50C460546FFF7C9FFA04210D305F1EE
:101FF0000800FFF7BDFF04446868BFF35B8FB4FBC4
:10200000F0F100FB1144AC60BFF35B8F012038BDE1
:102010000020FCE72DE9F041144607460D46FFF786
:10202000C5FF844228BF0446D4B1B84658F80C6BAB
:102030004046FFF79DFF06442E6040467E68FFF74E
:1020400097FF331A9C4203D801206C60BDE8F081F1
:102050006B603B68A61B0644AB600220EE60F5E7B0
:102060002046F3E738B50C460546FFF79FFFA04230
:1020700010D305F10C00FFF77BFF04446868BFF341
:102080005B8FB4FBF0F100FB1144EC60BFF35B8F9E
:10209000012038BD0020FCE72DE9FF410F466946CD
:1020A00006466C46FFF7B6FF002504EBC008444522
:1020B00008D0626820687919FFF750F9636808341E
:1020C0001D44F4E729463046FFF7CCFF284604B00C
:1020D000BDE8F081F8B505460C300F46FFF748FF24
:1020E00005F1080604463046FFF742FFA04230469D
:1020F00088BF6C68FFF73CFF201A386020B130467B
:102100002C68FFF735FF2044F8BD0000F7B51746EF
:1021100006460D46FFF732FFB842044628BF3C464C
:102120000190DCB1304601A9FFF7D4FF019B33B920
:102130003268C5E90233C5E9002401200CE09C4265
:1021400038BF01942860019884426860F5D9241A48
:1021500002203368EC60AB6003B0F0BD2046FBE7C3
:102160002DE9FF410E466946FFF7D0FF6C4600257A
:1021700004EBC007BC4209D0D4F804807019424671
:1021800054F8081BFFF7EAF84544F3E7284604B083
:10219000BDE8F08138B50546FFF7E2FF0446014689
:1021A0002846FFF71DFF204638BD0000EFF30983E6
:1021B000EFF30583044B9A6BDA6A9A6A9A6A9A6A11
:1021C0009A6A9A6A9B6AFEE700ED00E0EFF30983E2
:1021D000EFF30583044B9A6B9A6A9A6A9A6A9A6A31
:1021E0009A6A9B6AFEE700BF00ED00E0EFF3098307
:1021F000EFF30583034B5A6B9A6A9A6A9A6A9A6A52
:102200009B6AFEE700ED00E0FEE700000FB408B5B2
:10221000029801F09BF8FEE701F092BA01F06ABA69
:1022200001F068BA30B5094D0A4491420DD011F859
:10223000013B5840082340F30004013B2C4013F0BD
:10224000FF0384EA5000F6D1EFE730BD2083B8EDFC
:102250004FF0FF33F7B500EB81061946DFF848C0B1
:10226000DFF848E0B0421BD050F8042B01AF0192D8
:10227000042217F8014B81EA046108240D46DB189B
:102280004941013C002DBCBF83EA0C0381EA0E01E9
:1022900014F0FF04F2D1013A12F0FF02E9D1E1E7B4
:1022A000D843C94303B0F0BD9336EAA9EBE1F0424D
:1022B0002DE9F041C56915B9C161BDE8F0814B68F0
:1022C000AC4623F06047C3F38A4616EA230638BFBC
:1022D0003E464FEAD37EC3F380782B465A68BEEB66
:1022E000D27F22F060440AD0002A18DAA40CB4424B
:1022F00017D19D420FD10D60DEE71346EEE7A742EE
:1023000007D102F08044C2F3807242450BD054B131
:10231000EFE708D2EDE7CCF800100B60CDE7B44250
:1023200001D0B442E5D81A689C46002AE5D119606C
:10233000C3E700002DE9F0474FF47F49089D01F005
:1023400007044FEAD508224405F0070500EBD10049
:10235000944201D1BDE8F08704F0070705F0070AB1
:1023600057453E4638BF5646111BC6F108068E42F9
:1023700028BF0E46E108415C08EBD50E13F80EC0ED
:10238000B94029FA06F721FA0AF1FFB28CEA0101F5
:1023900047FA0AF739408CEA010C03F80EC03444BE
:1023A0003544D5E7082341F2210280EA012001B239
:1023B0004000002980B203F1FF33B8BF504013F052
:1023C000FF03F4D17047000038B50C468D18A542C4
:1023D00000D138BD14F8011BFFF7E4FFF7E7000058
:1023E0000346006848B1026819891A60DA88013228
:1023F00092B29142DA8038BF1A81704770B50446B4
:102400000D4688B0202200216846FEF7B9FF20461D
:102410000495FFF7E5FF024658B16B46054608AE46
:102420001C4603CCB44228606960234605F10805C8
:10243000F6D1104608B070BD082817D909280CD06D
:102440000A280CD00B280CD00C280CD00D280CD04E
:102450000E2814BF4020302070470C2070471020F9
:1024600070471420704718207047202070470000E4
:10247000082817D90C280CD910280CD914280CD9E5
:1024800018280CD920280CD930288CBF0F200E20FA
:102490007047092070470A2070470B2070470C20B6
:1024A00070470D207047000010B54B6823B9CA8AE9
:1024B00063F30902CA8210BDC4681A681C60C36055
:1024C000438A013B43824A60EFE700002DE9F84F61
:1024D0001D46CB8A0F46C3F3090106298146924661
:1024E0000B4630D00020AAB207F119049EB2052E87
:1024F0001FFA80F80FD8904503F1010306D3FB8A39
:102500000A4462F309030120FB821AE01AF8006012
:102510000130E654EAE79045F1D21C23A1F1060B05
:10252000BBFBF3F203FB12BB7C681FFA8BF6002C9B
:1025300045D14846FFF754FF044638B978606FF03C
:102540000200BDE8F88F4FF00008E6E700260660BD
:1025500078604FF0000BADB2454510D90AEB080387
:10256000221D13F8011B08F101089155B1B21B2976
:102570001FFA88F82BD0454506F10106F1D8FB8AF1
:10258000C3F30902154465F30903BCE71C46013295
:1025900092B22368002BF9D1AB1F0B441C21B3FB73
:1025A000F1F301339BB29A42D3D2BBF1000FD0D1E9
:1025B0004846FFF715FF20B9C4F800B0BFE7012275
:1025C000E7E7C0F800B05E4620600446C1E7454535
:1025D000D5D94846FFF704FF08B92060AFE7C0F837
:1025E00000B0002620600446B6E700002DE9F04F59
:1025F00085B007469146CDE90113BDF83C50002A4D
:1026000000F08F802DB10E9B002B00F08A80072DEB
:1026100030D807F10C00FFF7E3FE044628B96FF04D
:102620000204204605B0BDE8F08F14220021FEF719
:10263000A7FE2A460E9904F10800FEF78FFE681CDB
:10264000C0B2FFF715FFFFF7F7FE207499F80020DE
:10265000431E9BB202F01F02234462F03F021A7233
:10266000019B384643F0004161602146FFF720FEA0
:102670000124D6E74FF000084FF0800A4646444652
:1026800000F10C0303930398FFF7AAFE834600288A
:10269000C5D014220021FEF773FE002E38D102208F
:1026A000029BABF808300E9B00F10802D2B29919D8
:1026B0005A440130C0B2082801D0AE422AD3FFF7F5
:1026C000D7FEFFF7B9FEAE4208BF4FF0400A99F8B7
:1026D0000020019B411E02F01F0242EA4812C9B2CB
:1026E0004AEA020A594443F0004281F808A08BF8F4
:1026F000100059463846CBF80420FFF7D9FD0134C5
:10270000AE424FF0000A24B288F00108BBD188E73E
:102710000020C8E711F801CB013602F801CBB6B2B0
:10272000C7E76FF001047CE7F8B5044615460E468E
:10273000282200211F46FEF723FE069BB5F5001F49
:102740006360079B28BF4FF6FF7223624FF00003C0
:1027500038BF6A09A76004F10C0097B29A4205D805
:102760000023036027826382A382F8BD06600133E1
:1027700030462036F2E7000003781BB94BB2002B3D
:10278000C8BF017070470000007870472DE9F74F0F
:10279000DDF83C90804692469B46BDF830500D9E39
:1027A0009DF83840BDF84070B9F1000F01D1002FFD
:1027B00051D11F2C4FD898F80000B0B9072F47D837
:1027C00035F0030347D13A4649464FF6FF70FFF70D
:1027D000FBFD20F001002D02400445EA0464400C9A
:1027E00044EA40244FF6FF7321E040EA0520072F1A
:1027F00040EA0464F6D900254FF6FF73C5F12000C6
:10280000A5F120022AFA05F10BFA00F001432BFA98
:1028100002F211431846C9B2FFF7C4FD0835402D36
:102820000346EBD13A464946FFF7CEFD0346324612
:1028300021464046CDE90097FFF7D8FE33780133B3
:10284000DBB21F2B88BF0023337003B0BDE8F08FCD
:102850006FF00300F9E76FF00100F6E72DE9F04FA4
:1028600085B0DDF84880924606469B460F9D9DF850
:1028700040209DF84490BDF84C70B8F1000F01D194
:10288000002F48D11F2A46D83378002B46D00C029F
:1028900044EA02649DF8381044EAC93444EA014429
:1028A0001C43072F44F0800432D900234FF6FF72F7
:1028B000C3F1200CA3F120002AFA03F10BFA0CFC5F
:1028C00041EA0C012BFA00F00143C9B21046039310
:1028D000FFF768FD039B02460833402BE8D13A46D8
:1028E0004146FFF771FD03462A4621463046CDE9B1
:1028F0000087FFF77BFEB9F1010F06D12B7801337A
:10290000DBB21F2B88BF00232B7005B0BDE8F08F12
:102910004FF6FF73E8E76FF00100F6E76FF0030092
:10292000F3E70000C06900B104307047C3691A685A
:10293000C261C2681A60C360438A013B4382704728
:102940002DE9F041D0F8188014461D464146002775
:10295000174E09B9BDE8F081D1E90223A21A65EB4F
:102960000303964277EB03031ED283698B420DD19A
:10297000FFF79AFD83691B688361C3680B60438A14
:10298000C1608169013B88464382E2E7FFF78CFD25
:102990000B68C8F80030C3680B60438AC160013B14
:1029A0004382D8F80010D4E788460968D1E700BF11
:1029B00080841E002DE9F04F8BB00D4614469B46D7
:1029C0008046DDF85090002800F01A81B9F1000F20
:1029D00000F01681531E3F2B00F21281012A03D111
:1029E000BBF1000F40F00C810023CDE90833B8F8AB
:1029F0001430B5EBC30F4FEAC30703D300200BB06D
:102A0000BDE8F08F2B199F42D8F80C3036BF7F1BE2
:102A10002746FFB21BB9D8F81030002B7BD02F2DE2
:102A20004ED8C5F13006B7424FF0000334BF3E46E2
:102A3000F6B2009329463246D8F8080008ABFFF7F3
:102A400079FCA7EB060A35445FFA8AFA3021B8F818
:102A5000143003F10053063BDB000493D8F80C302C
:102A60000393039B13B1BAF1000F2CD1D8F81000D7
:102A700040B1BAF1000F05D05246009608AB691A72
:102A8000FFF758FC38B2002FB8D066070AD00AAB5F
:102A900003EBD40111F8083C624202F00702134133
:102AA00001F8083C082C3DD9102C40F2B680202CAF
:102AB00040F2B880BBF1000F00F09D80082335E0A4
:102AC000BA460026C2E7049BE02B28BFE02306930A
:102AD0000B44AB42059315D95A1B924538BF524659
:102AE000039828BFD2B20096691A08AB0430079247
:102AF000FFF720FC079A1644AAEB020A1544F6B227
:102B00005FFA8AFA049B069A05999B1A0493039B21
:102B10001B680393A5E700933A462946D8F80800B6
:102B200008ABADE7BBF1000F13D00123B4EBC30F2B
:102B30006CD0082C12D89DF82030621E23FA02F2C5
:102B4000D50706D54FF0FF3202FA04F423438DF87F
:102B500020309DF8203089F8003050E7102C12D832
:102B6000BDF82030621E23FA02F2D10706D54FF0DD
:102B7000FF3202FA04F42343ADF82030BDF82030D0
:102B8000A9F800303BE7202C0FD80899631E21FAE2
:102B900003F3DA0705D54FF0FF3202FA04F40C43D1
:102BA0000894089BC9F8003029E7402C2BD0DDE9B8
:102BB0000865611EC4F12102A4F1210326FA01F186
:102BC00005FA02F225FA03F311431943CB0712D594
:102BD0000122A4F12003C4F1200102FA03F322FA36
:102BE00001F1A240524243EA010363EB4303324343
:102BF0002B43CDE90823DDE90823C9E90023FEE6DC
:102C00006FF00100FBE66FF00800F8E6082CA0D991
:102C1000102CB3D9202CEED8C3E7BBF1000FADD0F8
:102C2000022383E7BBF1000FBBD004237EE7000043
:102C3000012A30B5144638BF01220025402A28BF9A
:102C4000402285B0012CCDE9025517D81B788DF8AC
:102C5000083053070AD004AB03EBD20515F8083C43
:102C6000544204F00704A34005F8083C03460091D1
:102C700002A80021FFF75EFB05B030BD082CE5D9A6
:102C8000102C03D81B88ADF80830E2E7202C02D8BE
:102C90001B680293DDE7D3E90045CDE90245D8E79B
:102CA00010B5CB681BB98B600B618B8210BDC468FB
:102CB0001A681C60C360438A013B4382CA60F0E724
:102CC0002DE9F04FD1F8008093B018F0800FCDE9D6
:102CD0000323C8F3C01207BF4FF0020B1646C8F318
:102CE000C03BC8F30626B8F1000F04460D4680F23B
:102CF000D48118F0C043059340F0CF810B7B002BAB
:102D000000F0CB81BBF1020F03D00178B14240F05B
:102D1000C78108F07F0107917AB3C8F3074A2B44B3
:102D200093F80390760646EA0B4608F07F0246EADF
:102D300082465FEAD91346EA0A06069300F09180BC
:102D400000220023CDE90A2308F07F0300935246B6
:102D50005B46204667680AA9B84700287ED0A76965
:102D60009FB9314604F10C00FFF748FB0746E0B974
:102D70006FF0020013B0BDE8F08FC8F30F2A18F00F
:102D80007F0F08BF0AF0030AC9E73B699E420DD0D6
:102D90003F68002FF9D1314604F10C00FFF72EFBFC
:102DA00007460028E4D0A3693B60A7610026DDE95F
:102DB0000A234FF6FF70C6F1200E22FA06F103FA3D
:102DC0000EFEA6F1200C23FA0CFC41EA0E0141EAAA
:102DD0000C01C9B2083609920893FFF7E3FADDE95E
:102DE0000832402EE7D1B882FB7D09F01F06C3F3FD
:102DF00084039B1B98B2002BBCBF00F120031BB2C5
:102E0000D7E9022152EA0100C8F304680FD0039801
:102E1000821A049860EB0101A74890424FF000022B
:102E20008A4104D3069A002A5BD0012B23DDFA7D68
:102E30004FEA890302F0030203F07C031343FB759E
:102E400039462046FFF730FB069BA3B9FB7DC3F351
:102E50008402013262F38603FB7504E06FF00B001D
:102E600088E7A76917B96FF00C0083E73B699E42BA
:102E7000BAD03F68F6E719F0400F32D0039B142216
:102E8000BB60049B0021FB600DA8FEF779FA039B51
:102E900020460A93049BADF83EA00B932B1D0C9388
:102EA0002B7B8DF840B0013BDBB2ADF83C30079B8B
:102EB0008DF841608DF8433094F824308DF84280CD
:102EC00083F001038DF844300AA9A3689847FB7D7D
:102ED000C3F38403013303F01F039B02FB82002032
:102EE00048E7FB7DC9F34012B2EBD31F40F0DB8013
:102EF000C3F38403B34240F0D98006992B7B4FEA99
:102F00009912002934D0D20741D4032B40F2D1804A
:102F1000039BAE1DBB60049B3246FB602B7B394696
:102F2000033BDBB204F10C00FFF7D0FA00280DDA06
:102F300020463946FFF7B8FAFB7D0320C3F384032C
:102F4000013303F01F039B02FB8213E7AB883B8333
:102F50002A7B033AB88AD2B23146FFF735FAFB7DB5
:102F6000B882DA43C2F3C01262F3C713FB75B6E747
:102F70006AB92E1D013B32463946DBB204F10C0022
:102F8000FFF7A4FA0028D3DB2A7B013AE2E7F98AAB
:102F9000013BC1F309010529DAB25BD80023281DE2
:102FA00007F11A0C9A4208D910F801EB01330CF81A
:102FB00001E001310629DBB2F4D1934228BF00239E
:102FC000039938BF04330A91049938BFDBB20B91DF
:102FD00007F11A010C91796838BF5B190D910E93B6
:102FE000FB8AADF83EA0C3F309031A44079BADF872
:102FF0003C208DF8433094F824308DF840B083F0B5
:1030000001038DF8443000238DF841608DF8428033
:103010007B602A7BB88A013A291DFFF7D5F93B8BE3
:10302000B882834203D12046A3680AA99847204664
:103030000AA9FFF735FEFB7DB88AC3F38403013389
:1030400003F01F039B02FB823B8B984214BF1120AD
:1030500000208FE67B68002BAFD0062001E063469E
:103060001C30D3F800C0BCF1000FF8D1091A081DBC
:1030700005F1040C1844DDF814E09DF814308E447A
:10308000BEF11B0F99D89A4297D91CF8013B00F862
:10309000013B059B01330593EDE76FF0090069E6FD
:1030A0006FF00A0066E66FF00D0063E66FF00E0049
:1030B00060E66FF00F005DE680841E00EFF3098389
:1030C000203383F30988002383F3118870470000BD
:1030D000202080F3118862B60C4B0D4AD96821F488
:1030E000E0610904090C0A43DA60D3F8FC200949BD
:1030F00042F08072C3F8FC200A6842F001020A60C4
:103100001022DA7783F82200704700BF00ED00E05C
:103110000003FA05001000E0202310B583F31188A6
:103120000B4B5B6813F400630FD0EFF309844FF08F
:103130008073203CE36184F3098800F0B9F810B192
:10314000044BA36110BD044BFBE783F31188F9E73F
:1031500000ED00E07F05000882050008012209015A
:1031600000F1604303F56143C9B283F8001300F036
:103170001F039A4043099B0003F1604303F5614339
:10318000C3F880211A607047090100F16040C9B29C
:1031900000F56D40017670470022024BC3E9003311
:1031A0009A607047BC1E0020002382680374054BA0
:1031B0001B6899689142FBD25A68036042601060B4
:1031C00058607047BC1E002008B5202383F3118887
:1031D000037C032B05D0042B0DD02BB983F311886E
:1031E00008BD002243691A604FF0FF334361FFF7C7
:1031F000DBFF0023F2E7D0E9003213605A60F3E707
:10320000002382680374054B1B6899689142FBD8C0
:103210005A6803604260106058607047BC1E00200E
:10322000054B196908741868026853601A601861C0
:1032300001230374FDF792B9BC1E002030B54B1C6E
:1032400004460B4D87B010D02B690A4A01A800F044
:10325000FDF82046FFF7E4FF049B13B101A800F03E
:1032600011F92B69586907B030BDFFF7D9FFF8E7AE
:10327000BC1E0020C931000838B50C4D41612B69D6
:1032800081689A680446914203D8BDE83840FFF748
:103290008BBF1846FFF7B4FF01232C61014623744E
:1032A0002046BDE83840FDF759B900BFBC1E0020DC
:1032B000044B1A681B6990689B68984294BF002071
:1032C00001207047BC1E002010B5084C23682069FF
:1032D0001A6854602260012223611A74FFF790FF7C
:1032E00001462069BDE81040FDF738B9BC1E00203A
:1032F00008B5FFF7DDFF18B1BDE80840FFF7E4BFF0
:1033000008BD0000FFF7E0BFFEE7000010B50C4C61
:10331000FFF742FF00F08CF880220A49204600F0B7
:103320003DF8012344F8180C0374FFF7D1FE002385
:1033300083F3118862B6BDE81040034800F04EB830
:10334000E41E0020F84000080841000808B572B6E5
:10335000034B586200F0C8F900F060FAFEE700BFC6
:10336000BC1E002000F0A0B8EFF3118020B9EFF3ED
:103370000583202282F311887047000010B530B910
:10338000EFF30584C4F3080414B180F3118810BD71
:10339000FFF7AEFF84F31188F9E700008260022294
:1033A000028270478368A3F13C0243F80C2C026947
:1033B00043F83C2C426943F8382C074A43F81C2C4C
:1033C000C268A3F1180043F8102C022203F8082C5D
:1033D000002203F8072C70476D05000810B5202364
:1033E00083F31188FFF7DEFF00210446FFF744FF57
:1033F000002383F31188204610BD0000024B1B6997
:1034000058610F20FFF70CBFBC1E0020202383F360
:103410001188FFF7F3BF000008B50146202383F3AE
:1034200011880820FFF70AFF002383F3118808BDE5
:10343000054B03F11402C3E905224FF0FF32DA61B4
:1034400000221A62704700BFBC1E002010B5C0E900
:1034500003230B4A136A53699C68A1420CD85C6829
:10346000816003604460206058609868411A9960E8
:103470004FF0FF33D36110BD1B68091BECE700BFA1
:10348000BC1E0020036881689A680A449A604268FA
:1034900013605A6000234FF0FF32C360014BDA61C2
:1034A000704700BFBC1E002038B50F4C2246236A6F
:1034B0000133236252F8143F934206D020259A68C4
:1034C000013A9A6063699A6802B138BDD3E9001085
:1034D00001604860D968DA6082F31188186988470A
:1034E00085F31188EEE700BFBC1E00200C230360AB
:1034F0004FF0FF307047000000207047FEE70000EB
:10350000704700004FF0FF3070470000BFF34F8F4F
:10351000024AD368DB07FCD4704700BF002002409A
:1035200008B5074B1B7853B9FFF7F0FF054B1A6935
:10353000120641BF044A5A6002F188325A6008BD3F
:10354000C01F0020002002402301674508B5054B3D
:103550001B7833B9FFF7DAFF034A136943F080039E
:10356000136108BDC01F0020002002407F289ABFC1
:1035700000F58030C0020020704700004FF400606A
:1035800070470000802070477F2808B50BD8FFF7F0
:10359000EDFF00F500630268013204D1043083427C
:1035A000F9D1012008BD0020FCE700007F2838B5D4
:1035B000044623D8FFF7D8FEFFF7A8FFFFF7B0FFB8
:1035C000F3220F4B0546DA60022220461A61FFF70C
:1035D000CDFF58611A694FF4006142F040021A6150
:1035E000FFF794FF00F016F92846FFF7AFFFFFF74B
:1035F000C5FE2046BDE83840FFF7C6BF002038BDF5
:10360000002002402DE9F047044612F001000E466A
:10361000154606D040F2BD22234B1A600020BDE8BB
:10362000F087224BA2189A4204D940F2C2221E4BC4
:103630001A60F4E7FFF798FE4FF0010AFFF770FFFA
:10364000FFF764FFDFF868903146A61B012D88461E
:1036500006EB010705D8FFF779FFFFF78FFE012082
:10366000DDE7B8F80030C9F810A03B800024FFF770
:103670004DFFC9F810403B8831F8022B9BB29A42AB
:103680000FD040F2D922084B1A600A4B1F600A4B38
:103690001D600A4BC3F80080FFF758FFFFF76EFE6E
:1036A000BCE7023DD2E700BFBC1F002000000408B9
:1036B00000200240B01F0020B81F0020B41F0020CF
:1036C000084908B50B7828B11BB9FFF729FF01237A
:1036D0000B7008BD002BFCD0BDE808400870FFF758
:1036E00035BF00BFC01F00204FF480314FF00050A5
:1036F00000F092B870B5FFF737FE4FF47A710D4BBA
:103700000D4E1B6A326801FB03F3934237BF0B4A2D
:103710000A495168156836BF4C1CD1E90054546001
:103720005D1944F100043360FFF728FE2846214666
:1037300070BD00BFBC1E0020C41F0020C81F002099
:1037400070B5FFF711FE4FF47A710F4B0F4E1B6AE5
:10375000326801FB03F3934237BF0D4A0C495168AD
:1037600015683ABF4C1C5460D1E900545D1944F10E
:1037700000043360FFF702FE4FF47A7200232846FC
:103780002146FCF7F5FC70BDBC1E0020C41F0020C4
:10379000C81F002010B5094C013AD2B2FF2A00D14F
:1037A00010BD500854F82030013054F820009BB26E
:1037B00043EA004341F8043BEEE700BF046C0040DD
:1037C00010B50748013AD2B2FF2A00D110BD0C88CB
:1037D000530840F823404C88013340F82340F1E778
:1037E000046C004007B50122002001A9FFF7D2FFB9
:1037F000019803B05DF804FB13B50446FFF7F2FF30
:10380000A04205D00122002001A90194FFF7D8FFB2
:1038100002B010BD70470000704700007047000004
:1038200045F25552064B1A6002225A6040F6FF726A
:103830009A604CF6CC421A600122024B1A70704713
:1038400000300040D41F0020034B1B781BB14AF608
:10385000AA22024B1A607047D41F0020003000409B
:10386000044B1A682AB902F1804202F50432526A06
:103870001A607047D01F00204FF08072014B5A62CF
:10388000704700BF0010024008B5FFF7E9FF024B88
:103890001868C0F3407008BDD01F002008B5FFF7BE
:1038A000DFFF024B1868C0F3007008BDD01F002076
:1038B00070470000FEE700000A4B0B480B4A90429D
:1038C0000BD30B4BC11EDA1C121A22F003028B42DF
:1038D00038BF00220021FDF753BD53F8041B40F808
:1038E000041BECE7E84100086C2000206C2000205D
:1038F0006C2000207047000000F030B808B500F0E0
:103900006DF9FFF703FDBDE80840FFF7A9BF000010
:10391000704700004FF0FF310E4B1A6919611A69A8
:1039200000221A611869D868D960D968DA60DA6843
:10393000DA6942F08052DA61DA69DA6942F00062EB
:10394000DA61054ADB69136843F48073136000F0A1
:1039500025B900BF00100240007000401E4B1A68DD
:1039600042F001021A601A689007FCD55A6822F0EA
:1039700003025A605A6812F00C02FBD1196801F078
:10398000F90119605A601A6842F480321A601A68A4
:103990009103FCD54EF63162DA625A6842F4E812BD
:1039A0005A601A6842F080721A601A689201FCD557
:1039B0000A4A0B495A6012220A600A6802F007029A
:1039C000022AFAD15A6842F002025A605A6802F09A
:1039D0000C02082AFAD170470010024000641D0052
:1039E00000200240084A08B5516913680B4003F0F3
:1039F0000103536123B1054A13680BB1506898471E
:103A0000BDE80840FFF788BB00040140D81F002034
:103A1000084A08B5516913680B4003F0020353616B
:103A200023B1054A93680BB1D0689847BDE80840B8
:103A3000FFF772BB00040140D81F0020084A08B5F8
:103A4000516913680B4003F00403536123B1054A25
:103A500013690BB150699847BDE80840FFF75CBB9C
:103A600000040140D81F0020084A08B551691368B6
:103A70000B4003F00803536123B1054A93690BB16E
:103A8000D0699847BDE80840FFF746BB00040140F5
:103A9000D81F0020084A08B5516913680B4003F08D
:103AA0001003536123B1054A136A0BB1506A98475A
:103AB000BDE80840FFF730BB00040140D81F0020DC
:103AC000174B10B55A691C68144004F478725A6197
:103AD000A30604D5134A936A0BB1D06A98476006CF
:103AE00004D5104A136B0BB1506B9847210604D5CF
:103AF0000C4A936B0BB1D06B9847E20504D5094A89
:103B0000136C0BB1506C9847A30504D5054A936C10
:103B10000BB1D06C9847BDE81040FFF7FDBA00BF6D
:103B200000040140D81F00201A4B10B55A691C68C8
:103B3000144004F47C425A61620504D5164A136DA0
:103B40000BB1506D9847230504D5134A936D0BB103
:103B5000D06D9847E00404D50F4A136E0BB1506E38
:103B60009847A10404D50C4A936E0BB1D06E9847C8
:103B7000620404D5084A136F0BB1506F98472304B1
:103B800004D5054A936F0BB1D06F9847BDE810403C
:103B9000FFF7C2BA00040140D81F0020062108B573
:103BA0000846FFF7DBFA06210720FFF7D7FA0621C0
:103BB0000820FFF7D3FA06210920FFF7CFFA0621E4
:103BC0000A20FFF7CBFA06211720FFF7C7FABDE856
:103BD000084006212820FFF7C1BA000008B5FFF70A
:103BE00099FE044800F00AF8FFF792FEBDE808408D
:103BF00000F002B82041000800F042B80023194646
:103C00001C4A0133102BC2E9001102F10802F8D15D
:103C1000194B9A6942F07D029A619B690268174BC1
:103C2000DA6082685A6042681A60C26803F580638D
:103C3000DA6042695A6002691A608269C3F80C242A
:103C4000026AC3F80424C269C3F80024426AC3F8B4
:103C50000C28C26AC3F80428826AC3F80028026BE1
:103C6000C3F80C2C826BC3F8042C426BC3F8002CF5
:103C7000704700BFD81F002000100240000801401C
:103C80004FF0E023044A08215A6100229A6107227A
:103C90000B201A61FFF778BA3F19010008B52023FD
:103CA00083F31188FFF75EFB002383F3118808BDBF
:103CB00008B5FFF7F3FFBDE80840FFF72DBA000095
:103CC0000B460146184600F025B8000000F038B851
:103CD000012838BF012010B50446204600F028F81E
:103CE00030B900F007F808B900F00CF88047F4E7A5
:103CF00010BD0000024B1868BFF35B8F704700BF18
:103D000058200020062008B500F02CF90120FFF70C
:103D1000F5FB000010B504460448134620B10A46DE
:103D200002202146AFF3008010BD00BF000000005C
:103D3000024B0146186800F083B800BF1C08002041
:103D4000024B0146186800F033B800BF1C08002081
:103D500010B501390244904201D1002005E00378FA
:103D600011F8014FA34201D0181B10BD0130F2E73A
:103D70002DE9F0419BB10446C91A1778014403F1BB
:103D8000FF3C8C42204601D9002008E00578013430
:103D9000BD42F6D10CEB0405D618A54201D1BDE811
:103DA000F08115F8018D16F801EDF045F5D0E8E742
:103DB00038B50546002940D051F8043C0C1F002BB3
:103DC000B8BFE41800F0F2F81C4A136833B9636016
:103DD00014602846BDE8384000F0EEB8A34208D988
:103DE000206821188B4201BF19685B68091821609F
:103DF000EDE71A465B680BB1A342FAD91168501877
:103E0000A0420BD120680144501883421160E0D1D8
:103E100018685B68014411605360DAE702D90C232B
:103E20002B60D6E7206821188B4201BF19685B68B8
:103E30000918216063605460CBE738BD5C20002026
:103E4000F8B5CD1C25F0030508350C2D38BF0C2521
:103E5000002D064601DBA94203D90C233360002064
:103E6000F8BD00F0A3F821490A6814469CB9204F18
:103E70003B6823B92146304600F03CF838602946BB
:103E8000304600F037F8431C23D10C233046336012
:103E900000F092F8E3E723685B1B17D40B2B03D9E0
:103EA00023601C44256004E06368A2420CBF0B60E1
:103EB0005360304600F080F804F10B00231D20F021
:103EC0000700C21ACCD01B1AA350C9E72246646867
:103ED000CCE7C41C24F00304A042E3D0211A3046EE
:103EE00000F008F80130DDD1CFE700BF5C200020F2
:103EF0006020002038B50023054D044608462B609D
:103F0000FFF7F4FA431C02D12B6803B1236038BDDC
:103F1000642000201F2938B504460D4604D9162315
:103F200003604FF0FF3038BD426C12B152F82130BF
:103F30004BB9204600F030F82A4601462046BDE83D
:103F4000384000F017B8012B0AD0591C03D11623B2
:103F500003600120E7E70024284642F825409847FF
:103F60000020E0E7024B01461868FFF7D3BF00BF0F
:103F70001C08002038B50023064D044608461146AB
:103F80002B60FFF7BFFA431C02D12B6803B12360FB
:103F900038BD00BF64200020FFF7AEBA034611F819
:103FA000012B03F8012B002AF9D17047014800F0DA
:103FB00009B800BF68200020014800F005B800BF24
:103FC0006820002070470000704700006F72672E65
:103FD0006172647570696C6F742E61705F70657268
:103FE0006970685F5A75626178474E5353000000EC
:103FF0004E6F20617070207369670A00426164200F
:104000006677206C656E6774682025750A004261CA
:104010006420626F6172645F696420257520736833
:104020006F756C642062652025750A00426164200A
:1040300066772064657363726970746F72206C6553
:104040006E6774682025750A004261642061707093
:1040500020435243203078253038783A3078253064
:104060003878203078253038783A307825303878EC
:104070000A00476F6F64206669726D776172650A26
:104080000040A2E4F16468910600000042616420EF
:1040900043414E496661636520696E6465782E0010
:1040A0008000000000800000000080000000000090
:1040B0000000000031140008E51B0008491B00083F
:1040C0004114000871140008611600084514000826
:1040D00059140008491400084D140008551400082C
:1040E000511400088D1500085D140008491E0008D1
:1040F00069140008611500086D61696E0000000018
:1041000069646C650000000000410008001F002089
:10411000B01F00200100000009330008000000006B
:104120000C880000447B444444544424800E000026
:1041300044141114947B444400000000444444445B
:10414000444444440400000044424444444444443D
:1041500000000000444444444444444444C0FF7FBD
:104160000100000000000000ED030000000000005E
:10417000006803000000000040420F00FE2A01001A
:10418000D204000020080020000000000000000011
:10419000000000000000000000000000000000001F
:1041A000000000000000000000000000000000000F
:1041B00000000000000000000000000000000000FF
:1041C00000000000000000000000000000000000EF
:1041D00000000000000000000000000000000000DF
:0841E0000000000000000000D7
:00000001FF
